:02000000C72F08
:0A000600E508031D07280800F93083
:10001000FF3E031D0828E50B07280800FA30E5001D
:100020000320FA30E5000320FA30E5000320FA301F
:10003000E5000320CC0B0E2808008312031386155D
:10004000861108000230831203130605E80003102E
:10005000680CC3000800E808031930280615312889
:10006000061108006808E9000310690DE800023075
:100070006805E800FD300605E900680869048600A7
:100080000800640E0F3985001D20640885001D20BE
:100090000230E50003200800823083160313860037
:1000A00001308312E8002B2022204308E700E801FA
:1000B0002B200130E8003220803083168600831226
:1000C0006708C300080080308316031386000130E0
:1000D0008312E8002B20E8013220E8012B200800E1
:1000E00006106208013A03197A286208023A0319D5
:1000F0007F2889286308803EE40041208928E601A2
:100100006308403EE5000318E60A65088038E4000D
:1001100041200230E50003200800790883169B0087
:100120001C141A088312C3000800FB01FD01FC0126
:100130006308FE006408FF00FB19AC28621CA628B7
:100140007E08FC070318FD0A7F08FD07E20C031078
:10015000FE0DFF0DFB0A9C287C08C3007D08C4002F
:100160000800FB01FD01FC016B08FE00FF01FB190B
:10017000C7286C1CC1287E08FC070318FD0A7F08ED
:10018000FD07EC0C0310FE0DFF0DFB0AB7287C08E1
:10019000C3007D08C4000800E801E701E601E501AD
:1001A000E901691AEB280310E50DE60DE00DE10DFC
:1001B000E70DE80D63086802031DE0286208670286
:1001C000031CE9286208E7026308031CE803E8024D
:1001D0006514E90AD1286708C3006808C40008004C
:1001E00083120313E8012B20E80132200130E800DC
:1001F0002B200130E80032200800E1010830E20045
:10020000E3016308803A803C031D08296208003C32
:10021000031822296108E7000310670DE10001308F
:1002200060056104E1006008E7000310670CE0006E
:100230006308E400E2080319E4036203E2006408CF
:10024000E30001298030E200E3016308803A803C4A
:10025000031D2C296208003C031846296108E800A8
:1002600032206108E7000310670CE1000130E8006C
:100270002B20E8012B206208E5006308E60003104C
:10028000E60C650CE2006608E30025294C20080016
:10029000E601E501E401E301E701671A67290310BC
:1002A000E30DE40DDD0DDE0DE50DE60D60086602E3
:1002B000031D5C295F086502031C65295F08E502D0
:1002C0006008031CE603E6026314E70A4D2963088D
:1002D000C3006408C4000800DB015808303EA500D4
:1002E0000430DB005B08003C0318CC29772978290F
:1002F000D71F8D295609E0005709E100E00F812939
:10030000E10A0A30E200E301CC204309DC004409A1
:10031000DD00DC0F8C29DD0A99295608E00057081A
:10032000E1000A30E200E301CC204308DC0044088D
:10033000DD005C08303EDE008313203084005B0863
:1003400084075E088000A429A529D71FBA29560969
:10035000DD005709DE00DD0FAE29DE0A0A30DF00BE
:10036000E00148214309DC004409E100DC0FB92920
:10037000E10AC6295608DD005708DE000A30DF0012
:10038000E00148214308DC004408E1005C08D60095
:100390006108D700DB0372295608303EA000DB015C
:1003A0005B08053C031CED295B085A0783169B007C
:1003B00083128313203084005B08840700088316AF
:1003C0009A001C1555309D00AA309D009C149C1865
:1003D000E7291C118312DB0AD0290800E00160081C
:1003E000053C031C002A60085F07F9008D20831379
:1003F000203084006008840743088000E00AEF2969
:10040000250EF039F900FA01F90CF90CF90C790C08
:100410000F39B0007A08B100200EF039E100610E0A
:100420000F39E2001030E3002730E4009520430844
:10043000E8004408E900210EF039E500650E0F39A7
:10044000E200E830E3000330E40095204308E600D2
:100450004408E70066086807EF006708F0006908CD
:100460000318F00AF007220EF039EA006A0E0F397D
:10047000EB006430EC00B1204308ED004408EE00CE
:100480006D086F07F4006E08F50070080318F50A90
:10049000F507230EF039F100710E0F39EB000A3029
:1004A000EC00B1204308F2004408F300720874071E
:1004B000F7007308F80075080318F80AF807240E07
:1004C000F039F600760E0F397707F9007808FA0050
:1004D0000318FA0A7908C3007A08C40008005F0804
:1004E000E2006008E300702006146108E400412087
:1004F0000800DC015C08053C031CDF2A5608E2000A
:100500005C08053C5707E300702006145C08033ABA
:10051000031D8F2A2E30E4004120DC0ADE2A902AB7
:10052000912AD91FA62A5809E0005909E100E00FD5
:100530009A2AE10A0A30E200E301CC204309DD00F7
:100540004409DE00DD0FA52ADE0AB22A5808E000C1
:100550005908E1000A30E200E301CC204308DD0045
:100560004408DE005D08303EE4004120B72AB82A86
:10057000D91FCD2A5809DD005909DE00DD0FC12A37
:10058000DE0A0A30DF00E00148214309E1004409A6
:10059000E200E10FCC2AE20AD92A5808DD00590806
:1005A000DE000A30DF00E00148214308E100440892
:1005B000E2006108D8006208D900DC0A7A2A5608ED
:1005C000E2005C085707DF00DC0A5F08E3007020E8
:1005D00006142C30E40041205608E2005C0857075E
:1005E000DF00DC0A5F08E30070200614F72AF82A0F
:1005F000DB1F0D2B5A09E0005B09E100E00F012B26
:10060000E10A0A30E200E301CC204309DD0044099D
:10061000DE00DD0F0C2BDE0A192B5A08E0005B0808
:10062000E1000A30E200E301CC204308DD00440889
:10063000DE005D08303EE40041200800C218252B92
:10064000DC01DD01DE01DF01C214DB01DA0104306F
:100650005A025B0803182E2B0319302BDB1F312B9A
:10066000322B682B332B342BD71F452B5609E00038
:100670005709E100E00F3D2BE10A1030E200E301F1
:10068000CC204309E400E40A4F2B5608E000570849
:10069000E1001030E200E301CC204308E4008313C2
:1006A0005C3084005A08840764088000560EE0001D
:1006B0000F30E005570EE100F039E0040F30E1059E
:1006C0006008D6006108D700DA0F672BDB0A272BFA
:1006D00063205908E000FD205E0EF039E100610E54
:1006E0000F39E2005F0EF0396207E000FD205C0E7A
:1006F000F039E100610E0F39E2005D0EF03962075A
:10070000E000FD20CE30E000FD205808E000FD2094
:10071000F020F03083168500F03086000800831248
:100720000313CE0182308316860008308312CF0077
:10073000D0015008803A803C031DA02B4F08003C9C
:100740000318BA2B4E08D2000310520DCE00013010
:10075000E8002B20222043084E04CE00E8012B2085
:100760005008D100CF080319D1034F03CF0051081F
:10077000D000992B0130E80032204E08C300080059
:1007800083120313861106100530E50003200330A1
:1007900085001D200530E5000320023085001D2066
:1007A0000530E50003202830E40041200530E50055
:1007B00003200830E40041200530E50003200C3020
:1007C000E40041200530E50003200630E40041202C
:1007D0000800CE014E080F3C031CFE2B4C08E20023
:1007E0004E08E300702006144E084D07F9008D20D6
:1007F00037304302E4004120CE0AEA2BCE01080044
:1008000063204C08E000FD208F234308CD00F0203A
:10081000F03083168500F030860083124D08C30047
:1008200008008312031306100130E4004120023057
:10083000E50003200800CF01CE010130D000D10136
:10084000D301D201D401D5014008DF000B30E00014
:100850007F30E1006F222830E500032032082E02AD
:10086000DA00330A031833082F02DB0036085A0770
:10087000DC003708DD005B080318DD0ADD075C08D3
:10088000DE005D08DF000310DE0DDF0D0310DE0D5E
:10089000DF0D0310DE0DDF0D30085E07E0003108CC
:1008A000E1005F080318E10AE1076008D60061086B
:1008B000D7004108D8004C08D9001E23013083120C
:1008C000340603193508031D6A2C3208CE0033089C
:1008D000CF006E2C2E08CE002F08CF004008D60087
:1008E0000330D7004E08D8004F08D9003008DA008E
:1008F0003108DB0079224E08D6004F08D7003008B7
:10090000D8003108D9004D08DA006C211930E50013
:100910000320D008031D8F2CD1080319C22D060E09
:100920000F390E3A031D9C2CB501B401D401D50139
:100930000130D000D1010800060E0F39073A031D1F
:10094000062D4008DF000230E0007E30E1006F221B
:100950004008023A031DC12CBC08031DBA2CBD0877
:10096000031DBA2CD830AE000430AF000130BC00FB
:10097000BD01C02CFC30AE000830AF00BD01BC0191
:10098000FA2CB408031DFA2CB508031DFA2CBE0876
:10099000031DDE2CBF08031DDE2CF630AE00283010
:1009A000AF007830DF00EE214308B2004408B30006
:1009B000F030C1000130BE00BF01FA2C01303E060C
:1009C00003193F08031DF02CFC30AE000830AF00C7
:1009D000B301B201F030C1000230BE00BF01FA2CF9
:1009E000D830AE000430AF00B301B2017030C100A6
:1009F000BF01BE01FA30E50003204008DF000230ED
:100A0000E0002030E1006F22D101D001060E0F3945
:100A1000033A031D152DD4010130D5004008DF0035
:100A20000B30E0007330E1006F22060E0F39053AFB
:100A3000031D232D0130D4004008DF000B30E000FF
:100A40007330E1006F2280300505D600D9010030F7
:100A500056020319D90A060E0F39D700D8010D30F6
:100A600057020319D80A58085904DC00060E0F393A
:100A7000DA00DB010B305A020319DB0A5B085C0465
:100A8000DD0055085D04DE0054085E040319C12D25
:100A900040300505DF00E20100305F020319E20A81
:100AA000060E0F39E000E1010D3060020319E10A82
:100AB00061086204E3005408630403198C2DB8082C
:100AC000031D652DB90803197D2D01303406031966
:100AD0003508031D6F2DB20F6E2DB30A7C2D3A0819
:100AE0002E07E4003B08E5002F080318E50AE50798
:100AF0006408AE006508AF008B2DB00F802DB10AE1
:100B00000A30300603193108031D8B2DAE0F892DD5
:100B1000AF0AB101B001BF2DB808031D922DB9086D
:100B20000319AA2D0130340603193508031D9D2D24
:100B3000B2080319B303B203A92D3A082E02E40048
:100B40003B0A03183B082F02E5006408AE00650865
:100B5000AF00BF2DB0080319B103B0030030FF3060
:100B60003106031DBF2D3008FF3A031DBF2DAE080F
:100B7000031DBB2DAF03AE030930B000B101D1019D
:100B8000D001892C0130D000D10132082E02D600CC
:100B9000330A031833082F02D7005608D20057082B
:100BA000D3000B305302031DD72DB9305202031C62
:100BB000F52DD31BF52DB208031DE12DB308031944
:100BC000EF2D3208523ED6003308D7000330031809
:100BD000D70AD7075608AE005708AF00F32D52309A
:100BE000AE000330AF00B101B0015308033C031D58
:100BF000FB2D5208513C0318FF2DD31F192EB208AC
:100C0000031D052EB3080319132E3208B83ED60073
:100C10003308D7000B300318D70AD7075608AE00A1
:100C20005708AF00172EB830AE000B30AF00B1013F
:100C3000B0012E2C83120313C701C6010130C80076
:100C4000C9010630CA00F03083168500F0308600F6
:100C50004030810083128B01C0236830DF00EE2119
:100C60004308A6004408A7003008A8003108A900DE
:100C70007030DF00EE214308AA004408AB003008C2
:100C8000AC003108AD007830DF00EE214308B2003F
:100C90004408B3000130CC004030CD00E9230230DD
:100CA000CC005030CD00E9230230CC000E20C80823
:100CB000031D5D2EC9080319822E0130CC00CD0121
:100CC000E9230230CC001030CD00E9230130D600FA
:100CD0000330D7002608D8002708D9002808DA00F2
:100CE0002908DB0079220230D6000330D7002A0819
:100CF000D8002B08D9002C08DA002D08DB00792257
:100D0000C901C80132082602CE00330A031833088D
:100D10002702D10036084E07D2003708D300510809
:100D20000318D30AD3075208D4005308D500031080
:100D3000D40DD50D0310D40DD50D0310D40DD50D44
:100D400028085407DA002908DB0055080318DB0AD5
:100D5000DB075A08D6005B08D7004108D800C63028
:100D6000D9001E2383122A08CE002B08D1000310BD
:100D7000CE0DD10D0310CE0DD10D0310CE0DD10D22
:100D80002C084E07D2002D08D30051080318D30AAF
:100D9000D3075208D6005308D700F030D800C0302F
:100DA000D9001E23C7308312CC0000244308C5009D
:100DB000FF3A031DDE2E3F30C500E52E451FE32E12
:100DC0002A30C500E52E2130C5000130DF000C308F
:100DD000E0004508E1006F22C130CC000024430848
:100DE000C500FF3A031DF72E3F30C500042F451FF5
:100DF000FF2E831605122A308312C500042F831696
:100E0000051621308312C5000230DF000C30E000EF
:100E10004508E1006F22060E0F39CB00073A03198F
:100E2000222F4B080B3A0319572F4B080C3A031982
:100E3000822F4B080D3A0319A92F4B080E3A0319BC
:100E4000C32FC32F11240130CC002030CD00E92363
:100E5000B808031D372FB908031D372F0130BA001A
:100E6000BB010630CA000130B800B901492F01307A
:100E7000380603193908031D462F0A30BA00BB0192
:100E80000A30CA000230B800B901492FCA01B901BD
:100E9000B8010130DF004A08E0002330E1006F2292
:100EA0000130CC000E200130C800C901C32F2A0830
:100EB000AE002B08AF002C08B0002D08B1000230A6
:100EC000C0003208C6003308C700B301B201B70141
:100ED000B601C030CC007030CD001B242E08AA0013
:100EE0002F08AB003008AC003108AD004608B20056
:100EF0004708B300E030B6000130B7000130C80049
:100F0000C901C32F2708273C031D882F2608103C42
:100F10000318A82FA71BA82F11240130CC003030B4
:100F2000CD00E9232608AE002708AF00B101B001CB
:100F30000130B400B5010130C0000130B800B90182
:100F4000C630CC007830CD001B240130C800C90168
:100F5000C32F2608AE002708AF002808B0002908D4
:100F6000B1000130C000C630CC006830CD001B2479
:100F70002E08A6002F08A7003008A8003108A900F5
:100F80000130C800C9013230E5000320572E83121A
:100F900003134210C210F630A6002830A700A901A2
:100FA000A801A030AA000230AB00AD01AC01AF0136
:100FB000AE01B101B001B830B2002430B300B501C8
:100FC000B401E030B6000130B7000130B800B9011B
:100FD0000130BA00BB010130BC00BD010130BE00D0
:100FE000BF010130C000F030C1008A110A121A2E70
:0A4000000200020003000B000000A4
:02400E0050025E
:104200008900AF005700570057005700570057006C
:104210005700570057005700570084007F00B10037
:104220008B00AF005700570057005700570057004A
:104230005700570057005700570084007F00B10017
:104240005700670065006800840057005700680049
:104250008400570057006800670084007F00B100A9
:10426000860083005700570057005700570057003B
:104270005700570057005700570084007F00B100D7
:1042800080008E00690083007D007B00570078006D
:104290008B008D005700640089008B008F00640044
:1042A0008A008E00570089009C00A300650057001B
:1042B00069006500690065006A00570067006C00CE
:1042C0002D002D002D002D002D002D002D002D0086
:1042D000310030003400380036003000FF00FF00AD
:1042E000300031003200340030003000FF00FF00A9
:1042F000300039003400300030003000FF00FF0093
:00000001FF
